:100000000128831686018312861206138613BC26E6
:020010000828BE
:100D7800F0010613861286130430F200E430F10005
:100D8800F10BC42EF20BC42E64001230F000700375
:100D9800013EF1001830F2004130F3000530F40054
:100DA8000030F501DC2E0310F50CF40CF30CF20CFA
:100DB800F103031DD72E721CE52E8312031386162A
:100DC800E82E8312031386120430F200E430F10097
:100DD800F10BEC2EF20BEC2E6400831203130617B2
:100DE8000430F200E430F100F10BF82EF20BF82E8B
:100DF80064008312031306130430F200E430F10098
:100E0800F10B042FF20B042F6400F003031DCB2E0B
:100E18008312031386120430F200E430F100F10B60
:100E2800132FF20B132F64000430F200E430F100AA
:100E3800F10B1C2FF20B1C2F64008312031386176F
:100E48000430F200E430F100F10B282FF20B282FC8
:100E580064000430F200E430F100F10B312FF20BA2
:100E6800312F64000430F200E430F100F10B3A2F26
:100E7800F20B3A2F64008312031386130430F20036
:100E8800E430F100F10B462FF20B462F64000430DA
:100E9800F200E430F100F10B4F2FF20B4F2F6400FA
:100EA8000430F200E430F100F10B582FF20B582F08
:100EB80064001230F0007003013EF1008330F2004C
:100EC8009030F3000230F4000030F501702F031069
:100ED800F50CF40CF30CF20CF103031D6B2F721CD0
:100EE800792F8312031386167C2F8312031386121D
:100EF8000430F200E430F100F10B802FF20B802F68
:100F080064008312031306170430F200E430F10082
:100F1800F10B8C2FF20B8C2F640083120313061332
:100F28000430F200E430F100F10B982FF20B982F07
:100F38006400F003031D5F2F83120313861204302D
:100F4800F200E430F100F10BA72FF20BA72F640099
:100F58000430F200E430F100F10BB02FF20BB02FA7
:100F680064008312031386170430F200E430F100A2
:100F7800F10BBC2FF20BBC2F64000430F200E430FC
:100F8800F100F10BC52FF20BC52F64000430F200FD
:100F9800E430F100F10BCE2FF20BCE2F6400831258
:100FA800031386130430F200E430F100F10BDA2F5A
:100FB800F20BDA2F64000430F200E430F100F10B98
:100FC800E32FF20BE32F64000430F200E430F10069
:100FD800F10BEC2FF20BEC2F6400831203130613B2
:100FE800861286130430F200E430F100F10BFA2F78
:080FF800F20BFA2F640008005F
:02400E00B82FC9
:00000001FF
